:0E38A30000640005000100A00032000A0005CC
:1027D200C10B4101250101AB01011500410123009B
:1027E200C10AC1004100D00041010100011C00C129
:0D27F20003C182C108010C00011B00C101E0
:102A4A00E4F5231225169000D07403F0123799305A
:102A5A00095FC209900123E004F0E550D3940040D5
:102A6A000DD5500A1238BD7F0A7E00123898786256
:102A7A00E6600B16E6B40106200503123838122167
:102A8A00F0E553F47003E552F4600DAF53AE521201
:102A9A00028C74FFF552F553900125E0B405121229
:102AAA0008007D017C007F0C121ACD90012574016B
:102ABA00F07896E6D39403403CE4F61238D712072E
:102ACA0089E4F51AE51A25E0249EF9E7900126F033
:102ADA00601AE014F0E0FFFDE51A25E0249DF8767F
:102AEA000008A605EF7005AF1A12384F051AE51A45
:102AFA00C3940740CFE515700241591515740F2587
:102B0A0015F8E614601814602114603624FE602655
:102B1A00240570E1B204E4FDFF12369880D7122929
:102B2A0017E4FD7F0112369880CB120FF9E4FD7F7E
:102B3A000212369880BF1233A8E4FD7F0512369838
:0B2B4A0080B3E4FD7F0312369880AAE0
:10251600D2DA439B4075A303E4FD7F051236987516
:1025260080FF759850758921758780758DFD758B2F
:10253600FD758A04758CF7D28ED28CD2A943BF0260
:102546001234E3D2AFD2AC750A011238D7123894DE
:102556001238D71238941238D71238941238D71244
:1025660038941238D71238941238D7E4F50AF5247D
:10257600E52425E024D1F582E43400F583E4F0A3D4
:10258600F00524E524B418E8E4F524E52425E02440
:1025960073F582E43401F583E4F0A3F00524E52421
:1025A600B406E87B017A01797F7F0E1235F0EF7071
:1025B6000690017F7480F0E4F524AF24121800051C
:1025C60024E524C3940240F2E4FDFC7F63121ACD95
:1025D600E4900193F07B017A0179227F0D1235F0A8
:1025E600EF70069001227480F07B017A0179257FD5
:1025F6000C1235F0EF70087D01FC7F0C121ACD909D
:102606000125E0700E7D01FC7F0C121ACD9001258C
:102616007401F07D0E7C007F05121ACD7D1F7C00B3
:102626007F07121ACD7B017A0079D07F081235F028
:10263600E4FDFF123698E4FD7F02123698900125DC
:10264600E06402702EFD7F04123698E4F524E5243A
:1026560025E02402F582E43401F583E4F0A3F005D5
:1026660024E524B410E8900193E030E704D2068014
:0626760002C2060208008A
:03000B000233FAC3
:1033FA00C0E0C0F0C083C082C0D075D000C000C099
:10340A0001C002C003C004C005C006C007758A0413
:10341A00758CF7789606D20978AB06E6D394024003
:10342A000276011236C7D007D006D005D004D003E1
:10343A00D002D001D000D0D0D082D083D0F0D0E05A
:01344A00324F
:10384F00E515C39406500AAE150515740F2EF8A68C
:02385F0007223E
:10369800ED701FEF25E024A3F582E43438F583E4C8
:1036A80093FA740193FBEF25E0249DF8A60208A67F
:0F36B8000322EDEF25E0249DF8760008A60522F9
:103799009000D0E0FF7006439B4075A303EFC394EC
:0E37A900014002D20AEFC394034002D2002274
:070FF900D291C2900230A664
:10078900900125E070183004055317FE80034317C4
:10079900013003055317FD8021431702801C3004E3
:1007A900055317FE8003431701E508D3940040075A
:1007B90015085317FD8003431702858016E4FFEFE0
:1007C90025E024D1F582E43400F583E0FCA3E0D3ED
:1007D90094F4EC94014007E51713F5178008E51721
:1007E900C3134480F5170FBF08D53004045317BF4E
:0407F9002243174040
:0107FD0022D9
:1036C7007580FF78ABE624FE6014047021C2B7E56D
:1036D7000A6005E4F5A080038516A0D2B622C2B61B
:0F36E700E50A6005E4F5A080038517A0D2B7229D
:0438D700759FA72210
:043894007F507EC320
:0B389800EF1FAC0670011E4C70F62202
:101D4F0000C1814001C0804101C0804100C181407C
:101D5F0001C0804100C1814000C1814001C080416C
:101D6F0001C0804100C1814000C1814001C080415C
:101D7F0000C1814001C0804101C0804100C181404C
:101D8F0001C0804100C1814000C1814001C080413C
:101D9F0000C1814001C0804101C0804100C181402C
:101DAF0000C1814001C0804101C0804100C181401C
:101DBF0001C0804100C1814000C1814001C080410C
:101DCF0001C0804100C1814000C1814001C08041FC
:101DDF0000C1814001C0804101C0804100C18140EC
:101DEF0000C1814001C0804101C0804100C18140DC
:101DFF0001C0804100C1814000C1814001C08041CC
:101E0F0000C1814001C0804101C0804100C18140BB
:101E1F0001C0804100C1814000C1814001C08041AB
:101E2F0001C0804100C1814000C1814001C080419B
:101E3F0000C1814001C0804101C0804100C181408B
:101E4F0000C0C101C30302C2C60607C705C5C4044B
:101E5F00CC0C0DCD0FCFCE0E0ACACB0BC90908C8BB
:101E6F00D81819D91BDBDA1A1EDEDF1FDD1D1CDCAB
:101E7F0014D4D515D71716D6D21213D311D1D0101B
:101E8F00F03031F133F3F23236F6F737F53534F40B
:101E9F003CFCFD3DFF3F3EFEFA3A3BFB39F9F8387B
:101EAF0028E8E929EB2B2AEAEE2E2FEF2DEDEC2C6B
:101EBF00E42425E527E7E62622E2E323E12120E0DB
:101ECF00A06061A163A3A26266A6A767A56564A4CB
:101EDF006CACAD6DAF6F6EAEAA6A6BAB69A9A8683B
:101EEF0078B8B979BB7B7ABABE7E7FBF7DBDBC7C2B
:101EFF00B47475B577B7B67672B2B373B17170B09B
:101F0F00509091519353529296565797559594548A
:101F1F009C5C5D9D5F9F9E5E5A9A9B5B99595898FA
:101F2F00884849894B8B8A4A4E8E8F4F8D4D4C8CEA
:101F3F00448485458747468682424383418180405A
:0727FF000160000252FFFF20
:1034E300C2B2E47860F67862F6FB7A0079517F061F
:1034F3007EEF1238B1E551F46004E55170137B009F
:103503007A0079517F061235F0EF700F7551FE8006
:103513000AE551FD7C007F06121ACDE5516003B424
:06352300FF037551FE22BA
:0A38BD00C2B2E47860F67862F622E9
:0B17F500C20CD2B27F0A7E00023898BE
:03002300022DE0CB
:102DE000C0E0C083C082C0D075D000C000C006C0A3
:102DF00007209802C1767860E6C394325007E60651
:102E00002464F8A699C2987860E6FFB4010575506D
:102E100032806AEF6407703A7865E6FE6403600406
:102E2000EEB406089001927408F08051EEB4100BD5
:102E3000200D089001927408F08042EEB4100B78D7
:102E40006AE62409900192F080339001927432F086
:102E5000802B900192E0B5070B75500078627606E2
:102E6000D20D8019EFB403157865E6B4190F9001FF
:102E7000927406F08007309904C299D20CD007D022
:0C2E800006D000D0D0D082D083D0E03249
:1038380012238B500F7508051217F51238C712108E
:073848000012134C0238BD11
:10238B007866E6FE08E67C002400F527EC3EF52691
:10239B00900192E07860666002C3227864E6FFF4F5
:1023AB00600AEF65516005EF6002C3227865E66451
:1023BB0019707CFB7A0079647D041235298E248F89
:1023CB00257868E6FE08E67C002400FFEC3EFEEF75
:1023DB0065257003EE65246002C3227867E6FF185B
:1023EB00E6FEC39F4004AD078002AD06EEC39F40DF
:1023FB0004AF068000E551C39D4006E551D39F40D5
:10240B0002C3227896E6FF7E001235E61235AF7CCA
:10241B00007D14120DB98D28E4F529E529C3952803
:10242B00500B7F647E00123898052980EED32278FA
:10243B0065E6FF6403600CEF64066007EF641060F1
:10244B0002C3227865E6FD64067039C3E52794085C
:10245B00E5269400502E7867E6FFC394025009904E
:10246B000193E030E01EC322EFC3940450099001A6
:10247B0093E030E10FC322EFB40809900193E030F1
:10248B00E202C3227866E6FE08E67A002400FFEA41
:10249B003EFEEF640A4E703CEDB4030E1235AF7C7A
:1024AB00007D05120DB97863A6057863E6640160BB
:1024BB0002C3221235AF7C007D14120DB98D28E4B6
:1024CB00F529E529C39528500B7F647E00123898B7
:1024DB00052980EE7B007A007964900192E024FE5E
:1024EB00FD1235298E248F25900192E0FD2462F890
:1024FB00E6FE74632DF8E67C002400FFEC3EFEEF55
:0A250B00B52506EEB52402D322C365
:0125150022A3
:10134C00E4F52AF52B7865E6FDB4061FE4F52A745E
:10135C0064252AF8E6F5997F327E00123898123807
:10136C00D7052AE52AC3940840E522ED6403600200
:10137C00A1D17866E6FE08E67C002400F525EC3E5B
:10138C00F5247869E6F5287864E6F529F59912379D
:10139C00BA7865E6F529300CFD1237B7E52825E05B
:1013AC00F529300CFD1237B7E52AC395284002A168
:1013BC00B67E00E525252AFFEE3524FEEF64634E4C
:1013CC007016F529300CFD1237B7900193E0F52912
:1013DC00300CFD1237B7A1B27E00E525252AFFEEB1
:1013EC003524FEEF648C4E7010F529300CFD12374D
:1013FC00B7300CFD1237B7A1B27E00E525252AFFC8
:10140C00EE3524FEC3EF9464EE9400505DE52A257E
:10141C0025FF7B007A00792612344BEF7004F526F9
:10142C00F5277E00E525252AFFEE3524FEC3EF9433
:10143C005AEE94004005E4F5298004E526F52930A0
:10144C000CFD1237B77E00E525252AFFEE3524FE6C
:10145C00C3EF945AEE940040057529018004E527EA
:10146C00F529300CFD1237B7A1B2AF2A7E00E52565
:10147C00252ACFEE3524CF249CCF34FFFEC3EF9426
:10148C0018EE9400504E7E00E525252AFFEE3524FB
:10149C00FEEF25E0FFEE33FE74092FF58274003E5B
:1014AC00F583E0F529300CFD1237B77E00E52525D4
:1014BC002AFFEE3524FEEF25E0FFEE33FE74092FF4
:1014CC00F58274003EF583E0A3E0F529300CFD12A3
:1014DC0037B7A1B2AF2A7E00E525252ACFEE3524F9
:1014EC00CF24D4CF34FEFEC3EF94A0EE9400502E44
:1014FC008E2C8F2D7B007A007926753E01122D19CA
:10150C0040067526227527B8E526F529300CFD1204
:10151C0037B7E527F529300CFD1237B7A1B2AF2A42
:10152C007E00E525252ACFEE3524CF240CCF34FEC2
:10153C00FEC3EF9458EE9400505A8E2C8F2D7C00E5
:10154C007D0B120D648F2BEF75F00BA4FFC3E52DF3
:10155C009FFFE52C95F0FEEF25E0FFEE33FEE52B2B
:10156C0075F016A42420F582E43400F583E5822F6F
:10157C00F582E5833EF583E0F526A3E0F527E52625
:10158C00F529300CFD1237B7E527F529300CFD1283
:10159C0037B78012E4F529300CFD1237B7752901E5
:1015AC00300CFD1237B7052A61B4300CFD785FE6BC
:1015BC00F599C20C300CFD7861E6F599C20C300C33
:1015CC0002C16880F97865E664107038F52A746495
:1015DC00252AF8E6F529F599C20C300CFDAF291235
:1015EC0037BE1238D7052AE52AC3940640E0785F47
:1015FC00E6F599C20C300CFD7861E6F599C20C2029
:10160C000C5A80FB7865E66419705118E6F529F5DB
:10161C0099C20C300CFDAF291237BE1238D7786541
:10162C00E6F529F599C20C300CFDAF291237BE1224
:10163C0038D7855129852999C20C300CFDAF291258
:10164C0037BE1238D7785FE6F599C20C300CFD78AE
:0C165C0061E6F599C20C300CFD1238D785
:01166800225F
:10100000752D01C211E4F52F7866E6FE08E6F97C3D
:10101000002400FFEC3EFEF5288F297865E6640683
:101020006002417FC3EF9464EE940040022179E9AD
:10103000940150257869E6FDE4FF121ACD7868E640
:10104000FD7C007F01121ACD900193E04401F0FD78
:101050007C007F63121ACD41CC7867E6D3940350AD
:10106000277869E6FD7C007F02121ACD7868E6FDDC
:101070007C007F03121ACD900193E04402F0FD7CC6
:10108000007F63121ACD41CC7867E66408702A08A5
:10109000E6FE08E67C002400FDEC3EFC7F08121A08
:1010A000CD900193E04404F0FD7C007F63121ACDE3
:1010B0007869E69000D0F041CC7867E6FF6405706F
:1010C0000241CCEF6407700241CCEFB4061278699C
:1010D000E6FD7C00121ACD7869E6F551D21141CCBB
:1010E0007867E6FFB40D127869E6FD7C00121ACD30
:1010F0007869E6900122F041CC7867E6FFB40E12E1
:101100007869E6FD7C00121ACD7869E690017FF0DF
:1011100041CC7867E6FFB40C197869E6FD7C0012D3
:101120001ACD7869E6900125F0600241CC750A017C
:1011300041CC7867E6FFB410107869E6FD7C0012B8
:101140001ACD7869E6F52D41CC7867E6B40A1B78AC
:1011500063E66401600241CC7869E6FD7C007F06AD
:10116000121ACD7869E6F55141CC7867E6FF7869C7
:10117000E6FD7C00121ACD41CCC3E529942CE5286C
:1011800094014002410F7866E67F00FE08E67C008D
:101190002400FFEC3ECF249CF529EF34FFF528D343
:1011A000E5299418E5289400504208E6FE08E62454
:1011B00000F525EC3EF524D3E52594FFE524648075
:1011C0009483400241CC7866E6FE08E62400FFECFA
:1011D0003EFEEF25E0FFEE33FE74092FF58274002A
:1011E0003EF583E524F0A3E525F041CCE5296463D1
:1011F0004528600241CC7869E6752400F525FDACF0
:10120000247F63121ACD7869E6900193F041CCC334
:10121000E529943CE5289401400241CC7866E67FBC
:1012200000FE08E67C002400FFEC3ECF24D4F52924
:10123000EF34FEF52808E6FE08E62400F525EC3E2E
:10124000F524E528C313FEE529137802C333CE3312
:10125000CED8F92400F58274003EF583E5295401C7
:1012600025E0FFE433FEE5822FF582E5833EF5833A
:10127000E524F0A3E525F0852852852953804D7893
:1012800065E6641070467869E6F52C7866E6FE0837
:10129000E67C002400F529EC3EF528E4F52AF52B40
:1012A000C3E52B952CE52A940050211238D7AF2B9B
:1012B000EF25E0246CF8E6FD7C00EF786726FF124E
:1012C0001ACD052BE52B70D8052A80D4E52D647F37
:1012D0007036752E77AF2E1237D4E4F5267B007A60
:1012E000007927AF261235F0EF600DE42526FDE4E6
:1012F00034EEFCAF27120FDD0526E526D39410400F
:10130000DCC2AF759F8080FEE52DB4FF07C2AF75CC
:101310009F8080FE3011341238D7752E77AF2E1291
:1013200037D4E4F5267B007A007927AF261235F012
:10133000EF600DE42526FDE434EEFCAF27120FDD4F
:0B1340000526E526C3940B40DCC2111B
:01134B00227F
:0938C700786176FF785F76FF223C
:0737B700852999C20CAF291E
:1037BE00785FE66FFF901D4F93786166795FF7EF44
:0537CE00901E4F93F670
:0137D30022D3
:083529008B2A8A2B892C8D2DC1
:10353100752E00752FFF7DFFAF2D152DEF6026AB8A
:103541002A052CE52CAA2B7002052B14F9120CFA72
:10355100652FFF901D4F936D752E00F52FEF901E77
:0A3561004F93FD80D3E52FFEEDFF30
:01356B00223D
:03280600011F08A7
:1030A60012356CE51F139292E51FA2E19293A2E2FC
:1030B60092947FB1122FDE1236F6EF4E600302387D
:1030C600D07F017E0012389812362F8E1D8F1E1269
:1030D600374E7F017E0012389812362F8E248F25A8
:1030E60012374E7F017E0012389812362F8E268FA9
:1030F600271238D0E51E2525FFE51D35245403F596
:10310600288F29E51FB40815E527B52925E526B535
:1031160028207D0DAF25AE241216698015E527B54A
:103126002910E526B5280BE51F14FDAF25AE2412A0
:0E3136001669051FE51FD3940D4003751F0891
:013144002268
:10356C00C2B47F017E00123898D2B5D2B47F027EED
:10357C0000123898C2B57F057E00123898C2B47F0D
:10358C00027E00123898D2B5D2B47F027E00123877
:10359C0098C2B57F057E00123898C2B47F027E00B7
:0335AC000238984A
:10374E00E4FFFE20B50C0FBF00010EEF64644E7057
:10375E00F222D2B57F017E00123898D2B4C2B57F64
:0A376E00017E00123898D2B5C2B4F3
:01377800222E
:022FDE00AD073D
:102FE0007B08ED3392B5D2B47F017E00123898C2CF
:0E2FF000B47F017E00123898ED25E0FDDBE491
:012FFE0022B0
:10362F00E4F52AF52BFDD2B47F017E00123898E520
:10363F002B25E0FFE52A33FEA2B5E433FBEEF52A96
:10364F00EF4BF52BC2B47F017E001238980DBD0AE7
:05365F00D5AE2AAF2BDF
:013664002243
:0738D000C2B5D2B4D2B5224B
:1036F600E4F52AF52BFBFA20B510D2B47F017E0043
:10370600123898C2B47E007F00220BBB00010AEB80
:0B37160064324A70E2C2B47E007F0102
:013721002285
:061669008D2AAB07AA0662
:10166F00E52A25E024D1F582E43400F583E0FEA3DA
:10167F00E0FFC3EB9FFFEA9EFE123861D3EF946445
:10168F00EE648094804014E52A25E024D1F582E4AD
:10169F003400F583EAF0A3EBF0804CE52A25E02433
:1016AF00D1F582E43400F583E0FCA3E0C39BEC9A10
:1016BF0050107482252AF582E43401F583E004F09A
:1016CF008025E52A25E024D1F582E43400F583E076
:1016DF00FCA3E0D39BEC9A400E7482252AF582E49A
:1016EF003401F583E014F07482252AF582E4340185
:1016FF00F583E0FBD36480948A500AC3EB64809433
:10170F00764002E196D3EF9428EE64809480401CDB
:10171F007C007D05120DB9E52A25E024D1F582E480
:10172F003400F583EE8FF0120DEF804ED3EB648013
:10173F00948A4016E52A25E024D1F582E43400F599
:10174F0083E475F001120DEF8030C3EB6480947663
:10175F005028E52A25E024D1F582E43400F583E012
:10176F00FEA3E04E6014E52A25E024D1F582E4348F
:10177F0000F58374FFF5F0120DEF7482252AF582C0
:10178F00E43401F583E4F0E52A25E024D1F582E481
:10179F003400F583E0FEA3E0D39400EE94044013ED
:1017AF00E52A25E024D1F582E43400F5837404F0B2
:1017BF00A3E4F0E52A25E024D1F582E43400F58393
:1017CF00E0FEA3E0FFE4FCFD7B607AEAF9F8C312C8
:1017DF000FA45011E52A25E024D1F582E43400F559
:0517EF0083E4F0A3F00B
:0117F40022D2
:0B38B1008F828E83E493120D407F0194
:0138BC0022E9
:060FD700FEAD07FC7F33B4
:100FDD00AB0775F65575F6AA75F65543BF048CF437
:0C0FED00AF058FF58BF675F7807F0022B2
:1037D400C2AF75F65575F6AA75F65543BF04EF25C5
:0C37E400E0F5F4E4F5F575F782D2AF22B1
:063356008B4D8A4E894FE9
:10335C00120E05FBAAF0530201EB24FFFFEA34FF27
:10336C00FE7C007D0F120D64A905EB241DFFE43AD1
:10337C00FEE97C00C3EF9DFFEE9CFED3EF94FFEEC5
:10338C00940140037F0022C3740F9DFFE49CAB4D5E
:0B339C00AA4EA94F8FF0120E307F01E7
:0133A7002203
:063300008B478A48894951
:103306001238D7EF25E0F54A754B00854B82F583D9
:10331600E493B433037F0022054BE54B7002054A64
:10332600854B82854A83E493B4FF14AB47AA48A928
:1033360049E54A854BF0120E681238D77F01227B89
:0F334600007A00794A123356EF70D51238D7FF4C
:013355002255
:0E380000AF3F1238738F44FB7A007934AF303B
:0E380E00EF75F0148425E025442463020D407C
:0237F000AC0724
:0E37F200ED25E07B00FAAF04FC7D00020FDD48
:06388400AD36AC35E4FF97
:0A388A00ED2401FDE43CFC020FDD1B
:10387300AE07BE01037F0222BE02037F01227F0047
:013883002222
:0831CE007A007935AD33AF3012
:0831D6008F478B488A49894AA2
:1031DE001238D7ED25E0F54B754C00854C82F58302
:1031EE00E493B4FF037F0022054CE54C7002054BBF
:1031FE00854C82854B83E493FE740193FDEEB547B7
:10320E0017ED6014AB48AA49A94AE54B854CF0125C
:10321E000E681238D77F0122BEFF09BDFF06123895
:10322E00D77F00227B007A00794B123356EF70C0A5
:04323E001238D7FF6C
:013242002269
:083145007B007A007935AD33FF
:08314D008B408A4189428D4349
:10315500E4F546F5471238D7E54325E0FEE42401BA
:10316500FFE43EF5448F458545828544837401938C
:10317500FEBE3314AB40AA41A942E5448545F01291
:103185000E681238D77F0122BE770CE54745467099
:10319500068544468545477B007A007944123356B7
:1031A500EF70C4E5474546700CAD43FF1237F0128A
:1031B50038D77F0022AB40AA41A942E5468547F0B2
:0831C500120E681238D77F01D9
:0131CD0022DF
:102C3A007545007546007547397548007549007530
:0C2C4A004A387B007A007937AF36AE358F
:0A2C56008E408F418B428A4389446F
:102C60008F828E837401937002FF221238D78541C0
:102C700082854083740293F54B7F03E5412403FD75
:102C8000E43540FCEFC3940F50118D828C83E493A4
:102C9000B4FF080F0DBD00010C80E9BF0F0612380C
:102CA000D77F0022E54345446011854182854083FA
:102CB000E493AB42AA43A944120D40E54645476060
:102CC00041AB45AA46A947E4F5F0120E68E4F54C7D
:102CD000E54CC3954B502BAB45AA46A947120E05B0
:102CE00075F000120E68ED254CF582E43CF583E4A6
:102CF00093FFAB45AA46A947E48FF0120E30054C6E
:102D000080CEE549454A600BAB48AA49A94AE54B44
:082D1000120D401238D77F01BB
:012D18002298
:0A32A4008B388A39893AAD07AC0671
:1032AE008D828C837401937002FF221238D77F03B4
:1032BE00ED2403FDE43CFCEFC3940F50118D828C82
:1032CE0083E493B4FF080F0DBD00010C80E9BF0F1E
:1032DE00061238D77F0022E539453A600F8D828C71
:1032EE0083E493AB38AA39A93A120D401238D77F2E
:0132FE0001CE
:0132FF0022AC
:08344B008F2E8B2F8A3089318E
:103453007535017B007A007932853544AF2E1238F9
:103463000E7A0009AD32AF2E1231D6EF601F852FD1
:1034730045853046853147754800754900754A00D2
:103483007B007A007900AF34AE33022C560535E564
:0834930035D3940240BD7F0017
:01349B00220E
:0835F0008F308B318A328933E0
:1035F8007537017B007A007934853744AF3012384B
:103608000E7A0009AD34AF301231D6EF600DAB3110
:10361800AA32A933AF36AE350232A40537E537D31F
:06362800940240CF7F0078
:01362E002279
:102B5500AD347F771237F0853444AB3BAD32AC31C1
:022B6500AF308F
:082B67008F408C418D428B432D
:102B6F007B007A007945AD441231D6EF601BAD463C
:102B7F00AC45AF42AE41122E94EF700AAD46AC4554
:102B8F00FF12388A80037F01227B007A007945AFDC
:102B9F0044123300EF7015E54425E0F54575460006
:102BAF00FEAF46120FD81238D77F0022AE45AF4680
:102BBF00AD07AC06AF40120FDDE54375F002A4D3AD
:102BCF00940CE5F0648094805013E5462401FFE4F3
:102BDF003545FEAD07FC7F77120FDD800BE54624F0
:102BEF0001FFE43545120FD7E5462402FFE43545D2
:102BFF00FEAD07FCAF43120FDD7901E9D3954350CA
:102C0F0024AF42E542E546240FFDE43545FCE9FBE0
:102C1F00C3ED9BFDEC9400FC120FDDE541F5427511
:0A2C2F0041000980D61238D77F015A
:012C39002278
:082E8C00AD36AC35AF32AE31BA
:082E94008E478F488C498D4ADE
:102E9C0085494C854A4D854D82854C83740193B48C
:102EAC0033037F00221238D77402254DF54DE435DB
:102EBC004CF54C854D82F583E493F54B054DE54D72
:102ECC007002054CE4FD854D82854C83E493B4FF80
:102EDC0011EDD3940C500B054DE54D7002054C0DC6
:102EEC0080E4E54B75F002A4FFC3ED9FE5F0648030
:102EFC00F8748098500BE54A2401FFE43549120F11
:102F0C00D77901E9D3954B501DAF48E548E9FDC38E
:102F1C00E54D9DFDE54C9400FC120FDDE547F548B1
:0B2F2C007547000980DD1238D77F01D7
:012F37002277
:061ACD008F308C318D32D8
:101AD300E4F53EF53FD3E53294FFE531940040054C
:101AE300753B028003753B017D017B007A007933EE
:101AF3008D44AF3012380EE53325E0F535753600E9
:101B0300853682F583E4937005AF331237D4853677
:101B130082853583E493FFB4FF08743B2DF8E4F624
:101B23008012743B2DF8A605EFB477028D3FEFB416
:101B330033028D3E0DBD03B21238D7E53C701EE56E
:101B43003D701AFB7A007933754401AF3012380EB9
:101B5300AD337F771237F0853344022B5FE53C606A
:101B630006E53D60028176E53F7006E53E70028141
:101B730076E53F700281017B007A007933F544AF4B
:101B83003012380E1231CEEF6042122E8CEF60020B
:101B9300A14EAD36AC35FF12388A853344122B5F24
:101BA300EF6002A14E123800122B55123145EF702F
:101BB30002A14E122C3AEF7002A14E853444AB3889
:101BC300AD3AAC39AF37122B6702388485334412F0
:101BD3002B5FEF6002A14E123800122B55123145D4
:101BE300EF7002A14E122C3AEF7002A14E853444DD
:101BF300AB38AD3AAC39AF37122B670238847B0070
:101C03007A007933853E44AF3012380E1231CEEF6D
:101C13006031122E8CEF6002A14EAF3E12380212D9
:101C23002B55123145EF7002A14E122C3AEF700280
:101C3300A14E853444AB38AD3AAC39AF37122B677C
:101C4300023884AF3E1238738F447B001238081277
:101C53002B55123145EF7002A14E122C3AEF700250
:101C6300A14E853444AB38AD3AAC39AF37122B674C
:101C73000238847B007A007934853F44AF301238D0
:101C83000E7A0019853E44AF3012380E1231CEEF72
:101C93006063122E8CEF6002A14EFB7A007935ADA2
:101CA30034AF301231D6EF602C122E8CEF6002A1CC
:101CB3004E122B5C123145EF7002A14E122C3AEFFB
:101CC3007002A14E853444AB38AD3AAC39AF37120C
:101CD3002B67023884122B5C123145EF606D122C96
:101CE3003AEF6067853444AB38AD3AAC39AF37125D
:101CF3002B670238847B007A007935AD34AF30121C
:101D030031D6EF6026122E8CEF7040122B5C12310D
:101D130045EF6037122C3AEF6031853444AB38AD70
:101D23003AAC39AF37122B67023884122B5C12316D
:101D330045EF6017122C3AEF6011853444AB38AD90
:0B1D43003AAC39AF37122B671238841E
:011D4E002272
:03280900015E0766
:103665000205050506060606070707080809090AEB
:103675000B0C0C0D0E10121315171B1E252A2F36B9
:103685003A3B37312C26231E1D1818151513111119
:03369500100F0F04
:0E280C0041018F00015C00C10F420190012CC0
:10291700E4F526F527D290A29233FDA293E433FB88
:10292700A294E433FAE55D139292E55DA2E19293F6
:10293700A2E29294C2917FF47E01123898D291ED6F
:1029470024FF9292EB24FF9293EA24FF9294C29081
:10295700E55D0475F0068485F05D900125E0600271
:1029670021FB20020221FBE55D30E015900190E09C
:10297700FEA3E0FFC374E89FF52574039EF524804A
:102987000A900190E0F524A3E0F525C37407955D4F
:1029970025E024D1F582E43400F583E524F0A3E5AE
:1029A70025F090018FE064207044C202D208300FF6
:1029B7001B900191E02464F0900190E03400F0E076
:1029C700B40320A3E0B4E81BC20F8017900191E085
:1029D700249CF0900190E034FFF0E07002A3E070D7
:1029E70002D20FE490018FF0E50A6002150A900108
:1029F7008FE004F0E55D25E024D1F582E43400F5AD
:102A070083E0FEA3E0FF900122E0FD7C00EF2DFFB5
:102A1700EC3ECF2480F529EF34FFF52830100CADBC
:102A270029FCAF5D1230008E288F29C3E52864800A
:102A370094805005E4F528F529AF29AE28122F38E0
:022A47008FA757
:012A4900226A
:042F38008E2A8F2B23
:102F3C00E4F52C90366593752D00F52ED3E52E9582
:102F4C002BE52D952A4006E4FAFBFFFE22052CAF5B
:102F5C002CEF3395E0FE74652FF58274363EF583C5
:102F6C00E493F9252EF52EE4352DF52DD3E52E958C
:102F7C002BE52D952A4050E52E952BFFE52D952A16
:102F8C00FEE9C39FFBE49EFA7C007D0AAF03FE12B0
:102F9C000D52AA06AB07E9FD120DB9AA06AB077CC8
:102FAC00007D05120D527D0A120DB9AA06AB07AFB2
:102FBC002CEF3395E0FE7C007D05120D52EF2BFBC0
:102FCC00EE3AFAAF03FE22E52C7082FA7BFF7FFF0C
:012FDC00FEF6
:012FDD0022D1
:09281A00420173000041017F97A7
:1033A800E4FFEF25E02473F582E43401F583E47546
:1033B800F001120DEFEF25E02473F582E43401F5F6
:1033C80083E0FCA3E0C39458EC94024020EF25E08E
:1033D80024D1F582E43400F583E4F0A3F0EF25E08E
:1033E8002473F582E43401F583E4F0A3F00FBF06FB
:0133F800B123
:0133F90022B1
:1021F000E580543FF524900181E06524600890015A
:1022000080E004F0800C900180E0D394004003E073
:1022100014F0900180E0D3940A5002618AE4F0FB4C
:10222000900181E0FFA803088002C313D8FC540189
:10223000F9E524A803088002C313D8FC5401FAFF6F
:102240007E007C037DE8120D52EB25E024F1F5823F
:10225000E43400F583EEF0A3EFF0E96A7002617CEC
:10226000EA7002616CEB25E02473F582E43401F539
:1022700083E0FEA3E0D39464EE94004012EB25E0EB
:102280002473F582E43401F583E4F0A37464F090E0
:10229000017FE0FAD39480402AEA2480FFE434FFEF
:1022A000FEEB25E02473F582E43401F583E0FCA322
:1022B000E0FD120D527C007D64120D64EF2480F568
:1022C00025802CEAFFC374809FFFE49400FEEB2579
:1022D000E02473F582E43401F583E0FCA3E0FD1211
:1022E0000D527C007D64120D64C374809FF525EB54
:1022F00025E02473F582E43401F583E0FEA3E0FFDA
:102300007C007D0A120D52EF2525FFEC3ECF248084
:10231000CF34FFFEEB25E024D1F582E43400F583D1
:10232000EEF0A3EFF0EB25E024D1F582E43400F5E4
:1023300083E0FEA3E0FFD39400EE94F04012EB257F
:10234000E024D1F582E43400F583E4F0A3F0801CAE
:10235000C3EF94CFEE94034013EB25E024D1F58234
:10236000E43400F5837403F0A374FFF0EB25E0245C
:1023700073F582E43401F583E4F0A3F00BEB64061B
:0A23800060024120900181E524F085
:01238A002230
:030100001F000ECF
:10282300C11060B0002000000000000000000000A4
:102833000000000000000000000000000000000095
:102843000000000000000000000000000000000085
:102853000000000000000000000000000000000075
:102863000000000000000000000000000000000065
:102873000000000000000000000000000000000055
:102883000000000000000000000000000000000045
:102893000000000000000000000000000000000035
:1028A3000000000000000000000000000000000025
:1028B3000000000000000000000000000000000015
:1028C3000000000000000000000000000000000005
:1028D3000000000000006020000004010401040166
:1028E30004010401040104010401040104010401BD
:0A28F30004010401040104010401C2
:10080000E4F525F5251238D7E52575F014A4FF7B0E
:10081000007A007934753E01122D194048E525759E
:10082000F014A404FF7B007A007934753E01122D88
:10083000194032E52575F014A42402FF7B007A00EC
:100840007934753E01122D19401BE52575F014A46D
:100850002403FF7B007A007934753E01122D194084
:1008600004C21081EED210E52575F014A4FF7B00C0
:100870007A007934753E01122D19E5354534703C06
:10088000E52575F014A404FF7B007A007934753EE9
:1008900001122D19E52575F016A42420F582E43403
:1008A00000F583E534F0A3E535F0752602752701E0
:1008B000E4753364F532F531F53021B9E52575F08D
:1008C00016A42420F582E43400F583E4F0A3F0F5C7
:1008D00026752701753364F532F531F530E5257558
:1008E000F014A4FF7B007A007934753E01122D19B3
:1008F000AE34AF35E4FCFDAB33AA32A931A830D316
:10090000120FBA400221B6E47FE87E03FDFCA83056
:10091000120FBA400221B6C3E49535FFE49534FEC8
:100920001238618E288F29E52575F014A404FF7B09
:10093000007A007934753E01122D19C3E49535FF14
:10094000E49534FE1238618E2A8F2BE4FCFDAB3324
:10095000AA32A931A830120E87C004C005C006C053
:1009600007AE28AF29E4FCFDF8F9AA06AB07D007CB
:10097000D006D005D004120F128F2F8E2E8D2D8C05
:100980002CE52575F016A42420F582E43400F583C7
:1009900075F002E527120FCBEEF0A3EFF00527E587
:1009A000332464F533E43532F532E43531F531E49E
:1009B0003530F53001F0752602E52575F014A425D3
:1009C00026FF7B007A007936753E01122D19AE366E
:1009D000AF37E4FCFDAB33AA32A931A830D3120FF4
:1009E000BA40026189E47FE87E03FDFCA830120F63
:1009F000BA40026189E526C3941440026189E52565
:100A000075F014A4252624FEFF7B007A0079387542
:100A10003E01122D19C3E5379539FFE5369538FEAD
:100A20001238618E288F29E52575F014A425260437
:100A3000FF7B007A007936753E01122D19E5257588
:100A4000F014A4252614FF7B007A007938753E0146
:100A5000122D19C3E5379539FFE5369538FE123862
:100A6000618E2A8F2BE52575F014A4252624FEFF20
:100A70007B007A007936753E01122D19E52575F057
:100A800014A4252614FF7B007A007938753E0112E4
:100A90002D19AE36AF37E4FCFDAA06AB07C3E5332C
:100AA0009BFBE5329AFAE5319400F9E5309400F8C1
:100AB000AE2AAF2BE4120E87C004C005C006C007E3
:100AC000AE28AF29E4FCFDF8F9AA06AB07D007D0A1
:100AD00006D005D004120F12A804A905AA06AB0778
:100AE000E4FCFDEB2539F52FEA3538F52EED39F527
:100AF0002DEC38F52CE52575F016A42420F582E4BC
:100B00003400F58375F002E527120FCBE52EF0A334
:100B1000E52FF00527E5332464F533E43532F5326B
:100B2000E43531F531E43530F530E52575F014A4C0
:100B30002526FF7B007A007936753E01122D19407B
:100B4000067536037537FFAE36AF37E4FCFDAB33C1
:100B5000AA32A931A830D3120FBA500221CEE5260D
:100B60009414400221CE05260526E52575F014A42F
:100B70002526FF7B007A007936753E01122D19403B
:100B8000C67536037537FF80BEE526C39414500240
:100B900081EEE47FE87E03FDFCAB33AA32A931A8E5
:100BA00030D3120FBA400281EEE52575F016A42469
:100BB00034F582E43400F5837403F0A374FFF0E5A8
:100BC0002575F014A42526FF7B007A007936753E42
:100BD00001122D194005E4F536F537E53745367035
:100BE0002215261526E52575F014A42526FF7B0081
:100BF0007A007936753E01122D1940DFE4F536F59D
:100C00003780D8E52575F014A4252604FF7B007AEB
:100C1000007938753E01122D19E47FE87E03FDFC52
:100C2000AB33AA32A931A830D3120FBA400281EEF9
:100C3000C374E89537FF74039536FE1238618E2829
:100C40008F29C374E89539FF74039538FE12386113
:100C50008E2A8F2BAE36AF37E4FCFDAA06AB07C356
:100C6000E5339BFBE5329AFAE5319400F9E53094DF
:100C700000F8AE2AAF2BE4120E87C004C005C006F0
:100C8000C007AE28AF29E4FCFDF8F9AA06AB07D0EF
:100C900007D006D005D004120F12A804A905AA0691
:100CA000AB07E4FCFDEB2539F52FEA3538F52EEDE1
:100CB00039F52DEC38F52CE52575F016A42420F532
:100CC00082E43400F58375F002E527120FCBE52EA0
:100CD000F0A3E52FF00527E5332464F533E435323E
:100CE000F532E43531F531E43530F530811905253B
:090CF000E525C39408500201053A
:010CF90022D8
:063000008C2A8D2BAB07AA
:103006007A05EA75F064A4FFD3E52B9FE52A95F0CF
:1030160040030A80EDEA75F064A4FFC3E52B9FE543
:103026002A95F050031A80EDEB75F016A42420F5CE
:1030360082E43400F58375F002EA120FCBE0FEA3BA
:10304600E0FFEB75F016A42422F582E43400F58344
:1030560075F002EA120FCBE0FCA3E0C39FF52DEC5E
:103066009EF52CEA75F064A4FFC3E52B9FFFE52AC5
:1030760095F0FEAC2CAD2D120D527C007D64120D28
:1030860064EB75F016A42420F582E43400F583750C
:0F309600F002EA120FCBE0FCA3E02FFFEC3EFEAE
:0130A5002208
:10028C00EEC313EF13F52475F014A4F526E524251D
:10029C00E025E02400F582E43400F583E0FEA3E0E1
:1002AC00C39401EE94044002E188E52425E025E0A6
:1002BC002402F582E43400F583E0FEA3E0C394014C
:1002CC00EE94044002E188E5262412FF7B007A00BC
:1002DC007927753E01122D194006752704752801E2
:1002EC00E52864017004E52764046002A1C8752543
:1002FC0010E5262525FF7B007A007927753E011233
:10030C002D194006752704752801E525D394004066
:10031C002CE5289401E527940440221238D71525A2
:10032C001525E5262525FF7B007A007927753E01EA
:10033C00122D1940D575270475280180CDE525604F
:10034C0002817BE52864017004E5276404703AE5BA
:10035C002425E025E02400F582E43400F583E0FC5C
:10036C00A3E0FD7B01AF26123243E52425E025E016
:10037C002402F582E43400F583E0FCA3E0FDE526DD
:10038C0004FF7B01123243E15CE52425E025E024E7
:10039C0000F582E43400F583E0FEA3E0C39528EE7B
:1003AC0095275066E5262402FF7B01AD28AC271269
:1003BC003243E52604FF7B007A007927753E011253
:1003CC002D19E5262403FF7B01AD28AC27123243FF
:1003DC00E52425E025E02400F582E43400F583E0F3
:1003EC00FCA3E0FD7B01AF26123243E52425E0257A
:1003FC00E02402F582E43400F583E0FCA3E0FDE5A3
:10040C002604FF7B01123243E15CE52425E025E064
:10041C002400F582E43400F583E0FCA3E0FDD395E1
:10042C0028EC9527402AE5262402FF7B0112324353
:10043C00E52425E025E02402F582E43400F583E090
:10044C00FCA3E0FDE5262403FF7B01123243E15CB3
:10045C00E52425E025E02402F582E43400F583E070
:10046C00FCA3E0FDE52604FF7B01123243E15CE5D1
:10047C0026FD7C00AB24AF25121F4F4002E15CE54A
:10048C002425E025E02400F582E43400F583E0F532
:10049C002BA3E0F52CE5262525FF7B007A00792798
:1004AC00753E01122D19D3E528952CE527952B4087
:1004BC0053E525D39400404C1238D7E52625252446
:1004CC0002FF7B01AD28AC27123243E5262525041B
:1004DC00FF7B007A007927753E01122D19E5262540
:1004EC00252403FF7B01AD28AC27123243152515BB
:1004FC0025E5262525FF7B007A007927753E01121C
:10050C002D1980A2E5257071D3E528952CE527954A
:10051C002B4066E5262402FF7B01AD28AC27123266
:10052C0043E52604FF7B007A007927753E01122DE6
:10053C0019E5262403FF7B01AD28AC27123243E5D5
:10054C002425E025E02400F582E43400F583E0FC6A
:10055C00A3E0FD7B01AF26123243E52425E025E024
:10056C002402F582E43400F583E0FCA3E0FDE526EB
:10057C0004FF7B01123243E15C05250525E52425AA
:10058C00E025E02400F582E43400F583E0FCA3E0F0
:10059C00FDE5262525FF7B01123243E52425E025C8
:1005AC00E02402F582E43400F583E0FCA3E0FDE5F1
:1005BC0026252504FF7B01123243E15C1238D7E477
:1005CC00F525E5262525FF7B007A007927753E0168
:1005DC00122D19E52425E025E02400F582E43400F1
:1005EC00F583E0FEA3E0D39528EE9527401DE52585
:1005FC009414501705250525E5262525FF7B007A43
:10060C00007927753E01122D1980C8E525641470F8
:10061C0041E52425E025E02400F582E43400F5834F
:10062C00E0FCA3E0FDE526252524FEFF7B0112322C
:10063C0043E52425E025E02402F582E43400F5832B
:10064C00E0FCA3E0FDE526252514FF7B01123243D7
:10065C00E15CE525703FE52425E025E02400F582EA
:10066C00E43400F583E0FCA3E0FDE5262525FF7BC3
:10067C0001123243E52425E025E02402F582E4341E
:10068C0000F583E0FCA3E0FDE526252504FF7B01B6
:10069C00123243E15CE5262525FF7B007A007927A1
:1006AC00753E01122D19E526252524FEFF7B007AC7
:1006BC00007929753E01122D19E52425E025E02449
:1006CC0000F582E43400F583E0FCA3E0FDC3E528EB
:1006DC009DFFE5279CFEC3ED952AFBEC9529FAC3FB
:1006EC00EF9BEE9A502BE5262525FF7B011232431A
:1006FC00E52425E025E02402F582E43400F583E0CE
:10070C00FCA3E0FDE526252504FF7B011232438086
:10071C003FE52425E025E02400F582E43400F58350
:10072C00E0FCA3E0FDE526252524FEFF7B0112322B
:10073C0043E52425E025E02402F582E43400F5832A
:10074C00E0FCA3E0FDE526252514FF7B01123243D6
:10075C00E52425E025E02400F582E43400F58374DB
:10076C0004F0A37401F0E52425E025E02402F582D1
:0C077C00E43400F5837404F0A37401F071
:01078800224E
:061F4F008C2D8D2E8B2F5E
:101F5500EF24FEF530E52F25E025E02400F582E4A9
:101F65003400F583E0F531A3E0F532E530252EFFA9
:101F75007B007A007933753E01122D19E5326534FF
:101F85007004E5316533601EE530D39400401715C4
:101F9500301530E530252EFF7B007A007933753E0C
:101FA50001122D1980D6E530702DE53265347004A7
:101FB500E53165336002D322E52F25E025E02402D3
:101FC500F582E43400F583E0FCA3E0FDE52E04FF93
:101FD5007B01123243C322E52F25E025E02402F5DB
:101FE50082E43400F583E0FCA3E0FDE530252E0412
:071FF500FF7B01123243C320
:011FFC0022C2
:1028FD0044016D0200020048016500680069006630
:09290D00006744015D00020002B4
:0C37220014F5828E83E493FFAC3EAD3FB3
:10372E00AB07C2AF75F65575F6AA75F65543BF04CD
:10373E008CF4AF058FF58BF675F780D2AF7F002234
:10381C00C2AF75F65575F6AA75F65543BF04EF257C
:0C382C00E0F5F4E4F5F575F782D2AF2268
:0C377900E52575F002A42454F9E4FAFBE5
:10378500120E05F58285F083E4932402FFE4338F5E
:04379500F0020E3000
:02349C00A9077E
:10349E00E925E0245DF582E43401F583E0A3E0F54F
:1034AE003BE925E02454F8E6FE08E6FFE53B24025E
:1034BE00FDE433FCE925E02461F582E43401F58373
:1034CE00E0FAA3E0C39DFDEA9CFCD3EF9DEE9C4089
:0434DE0002D322C330
:0134E20022C7
:021800008F2532
:10180200EF25E0246DF582E43401F583E0F528A3A9
:10181200E0F529EF25E025E02465F582E43401F5C1
:1018220083E0A3E0F526EF25E025E02467F582E4D6
:101832003401F583E0A3E0F527E52625E0F52A75D6
:101842002B00E52725E0752CFFF52D752E00852B45
:1018520082852A83E4936455600221C2AB2CAA2DAF
:10186200A92E120CFA6455600221C2E52B2401FF55
:10187200E4352AFEE52525E02454F8A60608A60745
:10188200E52525E02454F8E6FE08E6F5828E83E499
:1018920093F46020E52525E02454F8E6FE08E6AA44
:1018A20006C3852D83852E829582EA958350051283
:1018B200377980CCE52525E02454F8E6FE08E6C316
:1018C200952BF530EE952AF52FE52E2401F9E43516
:1018D2002DFEAF01E52525E02454F8A60608A6074B
:1018E200E52525E02454F8E6FE08E6F5828E83E439
:1018F20093F46030AB2CE52E2529F9E52D3528FA35
:10190200C0038A838982E52525E02454F8E6FE088F
:10191200E6AA06F9C3D0E0E99582EA95835005125A
:10192200377980BCE52525E02454F8E6FE08E6ABCD
:101932002CAA2DA92EAC02AD01C39DFFEE9CFED3B5
:10194200EF9530EE952F503FAE02AF01EF2401FF2D
:10195200E43EFEE52525E02459F582E43401F583D1
:10196200EEF0A3EFF074712525F582E43401F583DE
:10197200E526F0AE2AAF2BAD07AC06E4FF12372EF8
:10198200EF7002416AC322E52B2401FFE4352AFEEF
:10199200E52525E02459F582E43401F583EEF0A330
:1019A200EFF074712525F582E43401F583E527F023
:1019B200AC2DAD2EE4FF12372EEF7002416AC32226
:1019C200852B82852A83E493B4552BE52B2401FFD2
:1019D200E4352AFEE52525E02459F582E43401F5B3
:1019E20083EEF0A3EFF074712525F582E43401F55E
:1019F20083E527F08072AB2CAA2DA92E120CFAB423
:101A0200552DAE02AF01EF2401FFE43EFEE5252590
:101A1200E02459F582E43401F583EEF0A3EFF0748B
:101A2200712525F582E43401F583E526F08039AE8F
:101A32002AAF2BAD07AC06ED2401FFE43CFEE52501
:101A420025E02459F582E43401F583EEF0A3EFF0AA
:101A520074712525F582E43401F583E527F07F557D
:101A620012372EEF6002C322E52525E02459F582C4
:101A7200E43401F583E0FEA3E0FFE52525E02454EC
:101A8200F8A60608A607E52525E02459F582E434E0
:101A920001F583E0FEA3E02529FFE5283EFEE525CA
:101AA20025E02461F582E43401F583EEF0A3EFF042
:101AB200E52525E02454F8E6FE08E6F5828E83E467
:0A1AC20093F4600512377980E7D332
:011ACC0022F7
:022000008F3B14
:10200200EF25E02459F582E43401F583E0FEA3E0F4
:102012008E3CF53D74712FF582E43401F583E025A1
:10202200E0F53E753F00E53B25E0246DF582E434A2
:1020320001F583E0FFA3E090018DCFF0A3EFF0E480
:1020420090018AF090018DE0C313FF90018AE0C3F2
:102052009F50201238D77471253BF582E43401F584
:1020620083E0FF90018AE0FEEF2EFF12381CE004AD
:10207200F080D1053FE53F7002053E853D82853CFB
:1020820083E493F47002211E1238D7853D82853C89
:1020920083740193FF607AF46077053DE53DAE3CC1
:1020A2007002053C14F5828E83E49390018BF0E07C
:1020B200123729EF60037F0122053FE53F700205D9
:1020C2003E053DE53DAE3C7002053C123722EF6015
:1020D200037F0122053FE53F7002053EE490018A3D
:1020E200F090018BE0FF90018AE0C39F508D053D87
:1020F200E53DAE3C7002053C123722EF60037F01E2
:1021020022053FE53F7002053E90018AE004F0801F
:10211200D07B007A00793C123785017DE53B25E0D2
:102122002454F8A63E08A63FE53B25E02459F58253
:10213200E43401F583E0C313FF90018CF0FD747168
:10214200253BF582E43401F583E025E0FEE53B25FD
:10215200E02459F582E43401F583EEF0A3E4F0744F
:1021620071253BF582E43401F583EDF0E53B25E092
:102172002459F582E43401F583E0FEA3E0FF9001E7
:102182008DE0FCA3E0FDEF2DFFEE3CFEE53B25E0FC
:102192002461F582E43401F583EEF0A3EFF0E53B30
:1021A20025E02459F582E43401F583E0FCA3E0FD47
:1021B2007F5512372EEF60037F01227471253BF5A4
:1021C20082E43401F583E07D0025E0FCE4FF123770
:1021D2002EEF60037F0122E53B25E02459F582E4DE
:0D21E2003401F583E475F001120DEF7F006C
:0121EF0022CD
:08267C008F3B8B3C8A3D893E37
:10268400E4F544F545E53F25E0245DF582E43401B5
:10269400F583E0A3E0F546E53F25E02459F582E41F
:1026A4003401F583E0FEA3E08E40F541053BE53FB0
:1026B40025E02454F8E6FE08E6FFE5462401FDE49F
:1026C40033FCE53F25E02461F582E43401F583E041
:1026D400FAA3E0C39DFDEA9CFCD3EF9DEE9C400170
:1026E40022854182854083740193FE653B6010E43A
:1026F40093F4600B7B007A00794012378580E2EE18
:10270400B53B0BE5412401F545E43540F544E53F8F
:1027140025E02454F8E6FE08E6FFFDAC06AF4612B9
:10272400372E8F42E5426002C322E53F25E0245460
:10273400F808740226F618E436F6E4F543E543C3D4
:1027440095465033E53F25E02454F8E6FE08E62597
:1027540043FFE43EFEAD07FCAB3CAA3DA93E8543E6
:1027640082758300120D13FF12372E8F42E54260EB
:1027740002C322054380C6AF467E00E53F25E02420
:1027840054F808EF26F618EE36F6E53F25E0245413
:10279400F8E6FC08E6FDEF2401FFEE33FEC3ED9FEF
:1027A400FFEC9EFEAD07FCAF3B12372E8F42E54295
:1027B4006002C322E54545446012AE44AF45AD070F
:0D27C400AC06E4FF12372EEF6002C322D3F3
:0127D10022E5
:082D19008F3A8B3B8A3C893D97
:102D2100E53E25E02459F582E43401F583E0FEA374
:102D3100E08E3FF540E4F541F542053A8540828554
:102D41003F83E493F46053E53E25E02461F582E49A
:102D51003401F583E0FCA3E0D39540EC953F403A84
:102D6100854082853F83740193653A7022E542452F
:102D7100416016E5422401FFE43541FEAD07FCE464
:102D8100FF12372EEF6002C322853F418540427B0F
:102D9100007A00793F12378580A2E5424541603DC6
:102DA100854282854183740293FFAB3BAA3CA93DD6
:102DB100E48FF0120E68AB3BAA3CA93D120E0575DB
:102DC100F000120E68854282854183740393FFAB44
:0E2DD1003BAA3CA93DE48FF0120E30D322C382
:012DDF0022D1
:043243008F358B3602
:10324700E4F537EDF539ECF5381238D7AF361234E7
:103257009C5025E537C3940A500CAF36122000EF77
:103267006004053780ED7F057E00123898E537C387
:10327700940A400122E4F537E537C3940A50147BDA
:10328700007A00793885363FAF3512267C40040531
:0C3297003780E5E537C3940A400122D3DC
:0132A3002208
:03000000020200F9
:0C020000787FE4F6D8FD7581AB02024760
:100CFA00BB010689828A83E0225002E722BBFE02F8
:090D0A00E32289828A83E493222A
:100D1300BB010CE58229F582E5833AF583E0225095
:100D230006E92582F8E622BBFE06E92582F8E222DF
:0D0D3300E58229F582E5833AF583E49322F9
:100D4000BB010689828A83F0225002F722BBFE0192
:020D5000F3228C
:100D5200EF8DF0A4A8F0CF8CF0A428CE8DF0A42EB5
:020D6200FE226F
:100D6400BC000BBE0029EF8DF084FFADF022E4CC73
:100D7400F875F008EF2FFFEE33FEEC33FCEE9DEC3C
:100D8400984005FCEE9DFE0FD5F0E9E4CEFD22ED82
:100D9400F8F5F0EE8420D21CFEADF075F008EF2FCC
:100DA400FFED33FD4007985006D5F0F222C398FDBD
:050DB4000FD5F0EA225A
:100DB900C2D5EC30E709B2D5E4C39DFDE49CFCEE55
:100DC90030E715B2D5E4C39FFFE49EFE120D64C35C
:100DD900E49DFDE49CFC8003120D6430D507C3E457
:060DE9009FFFE49EFE22C4
:100DEF00C5F0F8A3E028F0C5F0F8E582158270028F
:060DFF001583E038F0222C
:100E0500BB010A89828A83E0F5F0A3E022500687B8
:100E1500F009E71922BBFE07E3F5F009E31922897A
:0B0E2500828A83E493F5F074019322AD
:100E3000BB010789828A83020DEF500B09C5F02799
:100E4000F7C5F01937F722BBFE0D09F8E325F0F3DB
:100E5000C5F019E338F322F889828A837401932557
:080E6000F0C5F0F8E49338221C
:100E6800BB010A89828A83F0E5F0A3F0225006F7D5
:0F0E780009A7F01922BBFE06F3E5F009F31922D2
:100E8700E88FF0A4CC8BF0A42CFCE98EF0A42CFC0A
:100E97008AF0EDA42CFCEA8EF0A4CDA8F08BF0A488
:100EA7002DCC3825F0FDE98FF0A42CCD35F0FCEBE7
:100EB7008EF0A4FEA9F0EB8FF0A4CFC5F02ECD39AC
:0F0EC700FEE43CFCEAA42DCE35F0FDE43CFC2219
:100ED60075F008758200EF2FFFEE33FECD33CDCCD3
:100EE60033CCC58233C5829BED9AEC99E582984056
:100EF6000CF582EE9BFEED9AFDEC99FC0FD5F0D633
:100F0600E4CEFBE4CDFAE4CCF9A88222B800C1B95C
:100F16000059BA002DEC8BF084CFCECDFCE5F0CB9A
:100F2600F97818EF2FFFEE33FEED33FDEC33FCEBD3
:100F360033FB10D703994004EB99FB0FD8E5E4F98E
:100F4600FA227818EF2FFFEE33FEED33FDEC33FC7B
:100F5600C933C910D7059BE99A4007EC9BFCE99A6F
:100F6600F90FD8E0E4C9FAE4CCFB2275F010EF2FB4
:100F7600FFEE33FEED33FDCC33CCC833C810D707B4
:100F86009BEC9AE899400AED9BFDEC9AFCE899F8EF
:0E0F96000FD5F0DAE4CDFBE4CCFAE4C8F92282
:100FA400EB9FF5F0EA9E42F0E99D42F0EC6480C8C4
:060FB40064809845F02264
:100FBA00EB9FF5F0EA9E42F0E99D42F0E89C45F08D
:010FCA002204
:0C0FCB00A42582F582E5F03583F5832231
:1035AF00AC58AD59AE5AAF5B780FEFA2E2EC20E604
:1035BF0001B35D5E5FF47004FCFDFEFFEF13FFEEE1
:1035CF0013FEED13FDEC13FCD8E08C588D598E5A79
:1035DF008F5BEE547FFE228E588F59E4F55AF55BC0
:0135EF0022B9
:10386100C3EE6480948040028007C3E49FFFE49E1E
:02387100FE2235
:10020C00022A4AE493A3F8E493A34003F68001F294
:10021C0008DFF48029E493A3F85407240CC8C333F3
:10022C00C4540F4420C8834004F456800146F6DFC2
:10023C00E4800B01020408102040809027D2E47E59
:10024C00019360BCA3FF543F30E509541FFEE493B7
:10025C00A360010ECF54C025E060A840B8E493A37E
:10026C00FAE493A3F8E493A3C8C582C8CAC583CAA9
:10027C00F0A3C8C582C8CAC583CADFE9DEE780BE61
:0129160000C0
:00000001FF
